:02000000552881
:10000600831206180A280B308F0021308C008618C0
:1000160010280F308F0019308C000619162815305D
:100026008F0012308C0086191C2820308F000C306F
:040036008C00080032
:10003A00831205152130CC007630CD00CD0B232854
:10004A00CC0B2328000005112130CC007630CD00DE
:0C005A00CD0B2D28CC0B2D280000080039
:10006600831205140630CB001330CC00AD30CD0022
:10007600CD0B3B28CC0B3B28CB0B3B2800000000CC
:1000860085140630CB001330CC00AD30CD00CD0B3F
:100096004A28CC0B4A28CB0B4A2800000000051042
:0400A60085100800B9
:1000AA00FF3083168600850103203320013090003B
:1000BA0010080F02031C802801308D008E010E08E3
:1000CA00003C031D6A280D080C02031C79281D2018
:1000DA0000300E06031D73280C080D060319792833
:1000EA008D0A03198E0A6428332010080F06031993
:0800FA008028900A5D2880288F
:02400E00FA3F77
:00000001FF
